:020000040000FA
:1000000016EF00F0EA6A060EE96EEF500EE0010E00
:10001000016E006A002EFED7012EFBD74A0E006E3D
:10002000002EFED700D0EF2EF2D7000CF86AD09E3B
:10003000EA6AE96AC150C00B0F09C16E070EB46EBF
:10004000C150C00B0F09C16EC290C69A949E938096
:100050009392010EC66E000EC76ED190800ED56EC3
:10006000CD6A000ECA6E000ECB6EB16A070EB46E7A
:100070009250926E030E006E002EFED7B450A19CDB
:10008000B56A92908980640E066EBCDF929089906A
:0A009000640E066EB7DFF5D703001B
:020000040030CA
:0E0000003FC0390E008781000FC00FE00F4097
:00000001FF
